:100000000C942A000C9445000C9445000C94450077
:100010000C9445000C94BC010C94E9010C9414025E
:100020000C9445000C945A010C9445000C94450026
:100030000C9445000C9445000C9436030C94450038
:100040000C9445000C9445000C9445000C9445001C
:100050000C94450011241FBECFE5D4E0DEBFCDBF18
:1000600010E0A0E6B0E0E6E0FFE002C005900D92EF
:10007000A43AB107D9F711E0A4EAB0E001C01D929B
:10008000A030B107E1F70C94B1000C940000CF93BD
:10009000DF93CDB7DEB7E7E3F0E08FE18083E4E301
:1000A000F0E08EEF8083E1E3F0E084E08083E2E340
:1000B000F0E088E38083DF91CF910895CF93DF93C1
:1000C000CDB7DEB723970FB6F894DEBF0FBECDBF16
:1000D0008091B1008823E1F31092B10080E29EE4A8
:1000E0009093FD008093FC001B822FC08B81482FD2
:1000F00055278B819927880F991FFC01EC53FF4FDF
:10010000808191819C0128513C4FCA01880F991F21
:10011000FC01E451FF4F318320832091FC0030919A
:10012000FD008B819927880F991FFC01E451FF4F37
:1001300080819181A901481B590BCA019093FD0050
:100140008093FC008B818F5F8B838B81883070F272
:1001500023960FB6F894DEBF0FBECDBFDF91CF91CF
:100160000895CF93DF93CDB7DEB727970FB6F894F6
:10017000DEBF0FBECDBF0E9447000E9438010E9423
:1001800028030E9477031092EB0083ED92E0909396
:10019000BF008093BE0081E293E09093C100809302
:1001A000C00078948091A8008823E1F31092A80001
:1001B0000E9420060E945F040E94C70600C0809132
:1001C000AB00813021F41092AB000E94F5068091C3
:1001D000A900813041F41092A9008091EB0088239E
:1001E00011F40E945E008091A800813029F51092E0
:1001F000A8000E9467061A821CC080E690E00E9458
:10020000B1038A8199270E94FB0387E690E00E9450
:10021000B1038A819927880F991FFC01E451FF4F90
:10022000808191810E94FB030E94EC038A818F5F91
:100230008A838A81893008F38091A700813009F090
:10024000BECF1092A700BBCFCF93DF93CDB7DEB761
:10025000F894E9E5F0E089E180837894DF91CF912B
:100260000895CF93DF93CDB7DEB7DF91CF91089597
:10027000CF93DF93CDB7DEB7E3E5F0E082E0808394
:10028000EFE4F0E01082EEE4F0E082E08083EAE464
:10029000F0E084EF91E091838083E8E4F0E080ED8A
:1002A00097E091838083E9E5F0E089E18083DF9145
:1002B000CF9108951F920F920FB60F9211248F9332
:1002C000CF93DF93CDB7DEB78091B5008F5F80937A
:1002D000B5008091B500893029F481E08093AB00AE
:1002E0001092B5008091EA008F5F8093EA008091C0
:1002F000EA008732C9F581E08093A9001092EA00F4
:100300008091B4008F5F8093B4008091B4008530F9
:1003100029F41092B40081E08093AA008091B20089
:100320008F5F8093B2008091B200843641F41092C6
:10033000B20081E08093A60081E08093A8008091C4
:10034000B200823319F481E08093A8008091B30059
:100350008F5F8093B3008091B3008A3029F41092AC
:10036000B30081E08093A700DF91CF918F910F9030
:100370000FBE0F901F9018951F920F920FB60F92FD
:1003800011242F933F934F935F936F937F938F939A
:100390009F93AF93BF93EF93FF93CF93DF93CDB72B
:1003A000DEB7E091BE00F091BF000995DF91CF91DB
:1003B000FF91EF91BF91AF919F918F917F916F913D
:1003C0005F914F913F912F910F900FBE0F901F9013
:1003D00018951F920F920FB60F9211248F93AF931F
:1003E000BF93EF93FF93CF93DF93CDB7DEB7A2E335
:1003F000B0E0E2E3F0E080818B7F8C93A5E3B0E096
:10040000E5E3F0E080818D7F8C9381E08093B10003
:10041000DF91CF91FF91EF91BF91AF918F910F90AD
:100420000FBE0F901F9018951F920F920FB60F924C
:1004300011242F933F938F939F93AF93BF93EF9389
:10044000FF93CF93DF93CDB7DEB72297DEBFCDBF4B
:10045000A2E3B0E0E2E3F0E0808184608C93ECE41E
:10046000F0E011821082A8E4B0E08091A400992706
:10047000880F991FFC01E451FF4F808191811196F3
:100480009C938E938091A400882339F4A5E3B0E077
:10049000E5E3F0E0808182608C938091A400282FB6
:1004A00033273A83298389819A8182309105C1F16A
:1004B00029813A812330310554F489819A8100974A
:1004C00089F029813A8121303105D9F04EC08981E6
:1004D0009A818330910599F129813A81243031053F
:1004E000E9F143C0A8E3B0E0E8E3F0E08081806197
:1004F0008C93A8E3B0E0E8E3F0E0808181608C9326
:1005000034C0A8E3B0E0E8E3F0E080818E7F8C9314
:10051000A8E3B0E0E8E3F0E0808182608C9325C03E
:10052000A8E3B0E0E8E3F0E080818D7F8C93A8E35E
:10053000B0E0E8E3F0E0808184608C9316C0A8E32B
:10054000B0E0E8E3F0E080818B7F8C93A8E3B0E03B
:10055000E8E3F0E0808188608C9307C0A8E3B0E016
:10056000E8E3F0E08081877F8C938091A4008F5F27
:100570008093A4008091A400893010F01092A40010
:100580002296F894DEBFCDBFDF91CF91FF91EF911E
:10059000BF91AF919F918F913F912F910F900FBE7F
:1005A0000F901F901895CF93DF93CDB7DEB7809152
:1005B000B6009091B7000097B1F4E6E4F0E08081D6
:1005C00091819093BD008093BC00AEE4B0E0EEE476
:1005D000F0E080818F7B8C9381E090E09093B70076
:1005E0008093B6002BC0E6E4F0E080819181909387
:1005F000BB008093BA00AEE4B0E0EEE4F0E08081AE
:1006000080648C932091BA003091BB008091BC0033
:100610009091BD00A901481B590BCA019093B900E4
:100620008093B8001092B7001092B6008091B80085
:100630009091B9009093FF008093FE00DF91CF91DD
:100640000895CF93DF93CDB7DEB7DF91CF910895B3
:10065000CF93DF93CDB7DEB7E7E2F0E01082E6E2BA
:10066000F0E08FEE8083DF91CF9108951F920F927B
:100670000FB60F9211242F933F938F939F93EF9375
:10068000FF93CF93DF93CDB7DEB7E6E2F0E01082C1
:100690008091A5009927E4E2F0E020813181880F64
:1006A000991FFC01EC53FF4F318320838091A500FB
:1006B0008F5F8093A5008091A500883010F0109284
:1006C000A500E7E2F0E08091A5008083E6E2F0E09B
:1006D0008FEE8083DF91CF91FF91EF919F918F916A
:1006E0003F912F910F900FBE0F901F901895CF93B1
:1006F000DF93CDB7DEB7E9E2F0E080E18083E0E4AC
:10070000F0E01082EAE2F0E088E18083E0E4F0E0EB
:1007100086E88083EBE2F0E082EC8083DF91CF918A
:100720000895CF93DF93CDB7DEB721970FB6F89436
:10073000DEBF0FBECDBF8983EBE2F0E08081992759
:10074000807290700097C1F3ECE2F0E089818083C1
:1007500021960FB6F894DEBF0FBECDBFDF91CF91CB
:100760000895CF93DF93CDB7DEB726970FB6F894F1
:10077000DEBF0FBECDBF9E838D838D819E81DC0148
:10078000FD0101900020E9F73197CF018A1B9B0BF7
:100790009C838B831A8219820FC029813A818D81B3
:1007A0009E81F901E80FF91F80810E9491038981E0
:1007B0009A8101969A83898329813A818B819C81D0
:1007C0008217930750F726960FB6F894DEBF0FBE38
:1007D000CDBFDF91CF910895CF93DF93CDB7DEB733
:1007E00080916A000E94910380916B000E949103A6
:1007F000DF91CF910895CF93DF93CDB7DEB76697A2
:100800000FB6F894DEBF0FBECDBF9E8B8D8B8D894A
:100810009E894AE050E09E012F5F3F4FB9010E9440
:100820003E07CE0101960E94B10366960FB6F8947A
:10083000DEBF0FBECDBFDF91CF910895CF93DF9381
:10084000CDB7DEB722970FB6F894DEBF0FBECDBF8F
:100850008A8387E089831FC08A81482F5527898131
:10086000282F332727FD309581E090E0022E02C02B
:10087000880F991F0A94E2F7842395231816190606
:1008800024F481E30E94910303C080E30E9491035A
:1008900089818150898389818823F4F680916A0057
:1008A0000E94910380916B000E94910322960FB6E3
:1008B000F894DEBF0FBECDBFDF91CF910895CF93E7
:1008C000DF93CDB7DEB70E94980463E080E00E941A
:1008D000FC058CE690E00E949E0562E081E00E94AB
:1008E000FC0587E790E00E949E050E948E04E0E3ED
:1008F000F0E080819927807290700097C1F70E9484
:100900009804DF91CF910895CF93DF93CDB7DEB7F1
:100910008DE00E94D305DF91CF910895CF93DF93AF
:10092000CDB7DEB78CE00E94D305DF91CF9108955B
:10093000CF93DF93CDB7DEB781E00E94D305DF917F
:10094000CF910895CF93DF93CDB7DEB726970FB63B
:10095000F894DEBF0FBECDBF9E838D838AE090E00A
:100960009C838B831CC082E390E09A8389830EC0B2
:100970008D819E8101979E838D838D819E810097BD
:10098000B9F789819A8101979A83898389819A81AC
:10099000009799F78B819C8101979C838B838B8136
:1009A0009C81009701F726960FB6F894DEBF0FBE24
:1009B000CDBFDF91CF910895CF93DF93CDB7DEB751
:1009C00021970FB6F894DEBF0FBECDBF8983898112
:1009D000992781709070882341F0A5E3B0E0E5E3AA
:1009E000F0E0808180618C9307C0A5E3B0E0E5E38F
:1009F000F0E080818F7E8C9389819927827090703E
:100A0000009741F0A5E3B0E0E5E3F0E0808180628B
:100A10008C9307C0A5E3B0E0E5E3F0E080818F7D33
:100A20008C938981992784709070009741F0A5E399
:100A3000B0E0E5E3F0E0808180648C9307C0A5E33B
:100A4000B0E0E5E3F0E080818F7B8C93898199278A
:100A500088709070009741F0A5E3B0E0E5E3F0E026
:100A6000808180688C9308C0A5E3B0E0E5E3F0E006
:100A700090818FE789238C9321960FB6F894DEBF7F
:100A80000FBECDBFDF91CF910895CF93DF93CDB748
:100A9000DEB7A5E3B0E0E5E3F0E0808184608C930D
:100AA00081E090E00E94A204A5E3B0E0E5E3F0E07D
:100AB00080818B7F8C93DF91CF910895CF93DF93CB
:100AC000CDB7DEB722970FB6F894DEBF0FBECDBF0D
:100AD0008A838A8182958F70898389810E94DC0450
:100AE0000E9445058A810E94DC040E9445052296E9
:100AF0000FB6F894DEBF0FBECDBFDF91CF91089542
:100B0000CF93DF93CDB7DEB721970FB6F894DEBF52
:100B10000FBECDBF8983A5E3B0E0E5E3F0E08081BF
:100B200088608C9389810E945E0521960FB6F894A7
:100B3000DEBF0FBECDBFDF91CF910895CF93DF937E
:100B4000CDB7DEB724970FB6F894DEBF0FBECDBF8A
:100B50009C838B838B819C81DC01FD0101900020B3
:100B6000E9F73197CF018A1B9B0B8A8319820EC04C
:100B7000898199279C018B819C81F901E80FF91FDC
:100B800080810E94800589818F5F898399818A8114
:100B9000981770F324960FB6F894DEBF0FBECDBF42
:100BA000DF91CF910895CF93DF93CDB7DEB7219733
:100BB0000FB6F894DEBF0FBECDBF898381E090E011
:100BC0000E94A204A5E3B0E0E5E3F0E08081877F26
:100BD0008C9389810E945E05A5E3B0E0E5E3F0E037
:100BE000808188608C9321960FB6F894DEBF0FBE8B
:100BF000CDBFDF91CF910895CF93DF93CDB7DEB70F
:100C000023970FB6F894DEBF0FBECDBF8A836B83E8
:100C10008A81882319F48B81805889838A81813065
:100C200019F48B818054898389810E94D30523968E
:100C30000FB6F894DEBF0FBECDBFDF91CF91089500
:100C4000CF93DF93CDB7DEB781E090E00E94A2049E
:100C5000A5E3B0E0E5E3F0E08081877F8C9383E05B
:100C60000E94DC040E94450585E090E00E94A204F9
:100C700083E00E94DC040E94450581E090E00E9430
:100C8000A20483E00E94DC040E94450582E00E94E9
:100C9000DC040E94450581E090E00E94A20488E205
:100CA0000E94D3058EE00E94D30581E00E94D30507
:100CB00084E890E00E949E056AE081E00E94FC05C5
:100CC00089E890E00E949E05DF91CF910895CF932F
:100CD000DF93CDB7DEB722970FB6F894DEBF0FBE15
:100CE000CDBF8091AC00882309F448C08091AF004B
:100CF000813009F041C08091AC00181634F4809125
:100D0000B0008F5F8093B00005C08091B00081502B
:100D10008093B0008091B00088231CF482E080931F
:100D2000B0008091B000833014F01092B000809138
:100D3000B000282F332727FD30953A8329838981F6
:100D40009A818130910579F029813A8122303105EB
:100D500079F089819A81009709F00EC060E080E007
:100D60000E94FC0509C069E080E00E94FC0504C007
:100D700060E081E00E94FC051092AC0022960FB664
:100D8000F894DEBF0FBECDBFDF91CF910895CF9312
:100D9000DF93CDB7DEB781E08093AF001092B00053
:100DA0000E94980460E080E00E94FC058EE890E0DC
:100DB0000E949E0569E080E00E94FC0586E990E0C3
:100DC0000E949E0560E081E00E94FC058DE990E0B4
:100DD0000E949E050E94840460E080E00E94FC0561
:100DE0001092AC00DF91CF910895CF93DF93CDB7F0
:100DF000DEB721970FB6F894DEBF0FBECDBF1982C4
:100E0000E0E3F0E08081992780719070009711F005
:100E100081E08983E0E3F0E0808199278870907019
:100E2000009721F0898193E08927898399818091B6
:100E30006900292F281B822F89838981992787FDA3
:100E4000909581709070882381F080916900982F2F
:100E50008981890F809369008981982F9270809190
:100E6000AC00890F81508093AC0021960FB6F894A6
:100E7000DEBF0FBECDBFDF91CF910895FB019F0173
:100E8000E8944230C4F04532B4F44A3029F497FB78
:100E90001EF4909581959F4F642F77270E946F07CE
:100EA000805D8A330CF0895D8193CB010097A1F7B7
:100EB00016F45DE251931082C9010C945F07DC01C6
:100EC000FC0101900020E9F73297AE17BF0730F41C
:100ED0007C916081708331976D93F7CF0895AA1B41
:100EE000BB1B51E107C0AA1FBB1FA617B70710F015
:100EF000A61BB70B881F991F5A95A9F78095909547
:060F0000BC01CD010895C3
:100F06004B2000000000003D00010D0A4550492D10
:100F16005465737465720056657273696F6E20301E
:100F26002E3264006875687500416B6B7500505011
:100F36004D2D4F75740050504D2D496E00444D583F
:040F46002D496E00C3
:00000001FF
